:020000040000FA
:0408000005EF06F00A
:1008100003B20FEF05F0F2B42AEF05F09EB032EF0D
:1008200005F09EB23AEF05F0F2A81AEF04F0F2B22A
:100830001CEF04F0E3EF05F0CD90F2929EA026EFBE
:1008400004F00101463F26EF04F0472B81C185F1FA
:1008500082C186F183C187F184C188F17DC181F1B4
:100860007EC182F17FC183F180C184F179C17DF1C4
:100870007AC17EF17BC17FF17CC180F175C179F1D4
:1008800076C17AF177C17BF178C17CF171C175F1E4
:1008900072C176F173C177F174C178F16DC171F1F4
:1008A0006EC172F16FC173F170C174F169C16DF104
:1008B0006AC16EF16BC16FF16CC170F1CECF69F19D
:1008C000CFCF6AF146C16BF147C16CF1CF6ACE6AF6
:1008D0000101466B476B9E90CD800EBC0E8E0EBA0A
:1008E00075EF04F00E8AE3EF05F00E8C0EBEB1EF4B
:1008F00004F069C16DF16AC16EF16BC16FF16CC139
:1009000070F16DC171F16EC172F16FC173F170C19F
:1009100074F171C175F172C176F173C177F174C16F
:1009200078F175C179F176C17AF177C17BF178C13F
:100930007CF179C17DF17AC17EF17BC17FF17CC10F
:1009400080F17DC181F17EC182F17FC183F180C1DF
:1009500084F181C185F182C186F183C187F184C1AF
:1009600088F10101516B526B536B546B69515127E4
:100970006A5152236B5153236C5154236D515127AB
:100980006E5152236F51532370515423715151278B
:10099000725152237351532374515423755151276B
:1009A000765152237751532378515423795151274B
:1009B0007A5152237B5153237C5154237D5151272B
:1009C0007E5152237F51532380515423815151270B
:1009D00082515223835153238451542385515127EB
:1009E000865152238751532388515423D89054332E
:1009F000533352335133D8905433533352335133EA
:100A0000D890543353335233513369C151F16AC1D1
:100A100052F16BC153F16CC154F1E3EF05F0039255
:100A2000030103EE00F080517F0BE92604C0EFFFC5
:100A3000802B8151805D700BD8A48B820000805187
:100A4000815D700BD8A48B9281518019D8B4079026
:100A5000E3EF05F0F2940101383FE3EF05F0392BA5
:100A6000E3EF05F09E900101463FE3EF05F0472BD1
:100A7000E3EF05F09E92C3CF48F1C4CF49F1C282A3
:100A800007B465EF05F03AC13EF13BC13FF13CC10F
:100A900040F13DC141F151C155F152C156F153C12F
:100AA00057F154C158F1010148514E2749514F2384
:100AB000E86A50230D2E65EF05F04FC14AF150C191
:100AC0004BF14E6B4F6B506B078E0201002FE3EF23
:100AD00005F03C0E006F01015D6776EF05F05E6783
:100AE00076EF05F05F6776EF05F060677AEF05F067
:100AF000AAEF05F061C100F162C101F163C102F129
:100B000064C103F10101010E046F000E056F000EB8
:100B1000066F000E076FC1EC12F000C161F101C158
:100B200062F102C163F103C164F100679FEF05F058
:100B300001679FEF05F002679FEF05F00367AAEFDB
:100B400005F05DC161F15EC162F15FC163F160C139
:100B500064F10E80D57ED5BE34D0D6CF3AF1D7CF52
:100B60003BF138C13CF1E86AE8CF3DF10F8001016B
:100B700047A7C7EF05F00E9A0E9C0E9E0101000ECE
:100B8000516F600E526F3D0E536F080E546F01018E
:100B90003ABFD7EF05F03B67D7EF05F03C67D7EFDB
:100BA00005F03D67D7EF05F0F288DCEF05F0F2982D
:100BB000516B526B536B546BD76AD66A0101386B19
:100BC000396BE3EF05F002C0E0FF005001C0D8FF31
:100BD0001000A6B2E9EF05F00CC0A9FF0BC0A8FFFA
:100BE000A69EA69CA684F29E550EA76EAA0EA76E80
:100BF000A682F28EA694A6B2FBEF05F01200A96EB3
:100C0000A69EA69CA680A8501200076A0E6A0F6ACC
:100C10000F010E0EC16E860EC06E030EC26E0F0166
:100C2000896A110E926E080E8A6EF10E936E8B6AAF
:100C3000800E946EF18E0D6A01014E6B4F6B506BFE
:100C40004A6B4B6B0F01280ED56EF28AB00ECD6E3B
:100C50009D800101516B526B536B546B556B566BFE
:100C6000576B586B596B5A6B5B6B5C6B0E9A0E9C97
:100C70000E9E760ECA6E9D8202013C0E006FCC6AFB
:100C8000160EFFEC05F0E8CF00F1170EFFEC05F0B3
:100C9000E8CF01F1180EFFEC05F0E8CF02F1190ED4
:100CA000FFEC05F0E8CF03F1010103AF72EF06F0AE
:100CB000B8EC13F0160E0C6E00C10BF0E9EC05F069
:100CC000170E0C6E01C10BF0E9EC05F0180E0C6E5E
:100CD00002C10BF0E9EC05F0190E0C6E03C10BF02C
:100CE000E9EC05F000C15DF101C15EF102C15FF107
:100CF00003C160F100C161F101C162F102C163F1A0
:100D000003C164F11A0EFFEC05F0E8CF00F11B0EF1
:100D1000FFEC05F0E8CF01F11C0EFFEC05F0E8CF89
:100D200002F11D0EFFEC05F0E8CF03F1010103AF66
:100D3000C8EF06F0B8EC13F01A0E0C6E00C10BF001
:100D4000E9EC05F01B0E0C6E01C10BF0E9EC05F0AF
:100D50001C0E0C6E02C10BF0E9EC05F01D0E0C6EC2
:100D600003C10BF0E9EC05F01A0EFFEC05F0E8CF3B
:100D700000F11B0EFFEC05F0E8CF01F11C0EFFECBB
:100D800005F0E8CF02F11D0EFFEC05F0E8CF03F10E
:100D900000C165F101C166F102C167F103C168F1EB
:100DA000240EAC6E900EAB6E240EAC6E080EB86EB8
:100DB000000EB06E1F0EAF6E0401806B816B0F01D1
:100DC000900EAB6E0F019D8A0301806B816BA26B4D
:100DD0008B9207900001F28EF28C07B085EF10F035
:100DE0000EB0C3EF0BF00301805181197F0BD8B413
:100DF00085EF10F013EE00F081517F0BE126812B7F
:100E0000E7CFE8FFE00BD8B485EF10F023EE82F0D7
:100E1000A2511F0BD926E7CFDFFFA22BDF50780AA4
:100E2000D8A485EF10F0078061C100F162C101F123
:100E300063C102F164C103F10101040E046F000EED
:100E4000056F000E066F000E076FC1EC12F000AFC9
:100E500033EF07F00101030E616F000E626F000EA9
:100E6000636F000E646F03018251720AD8B4C3EF3E
:100E70000BF08251520AD8B4C3EF0BF08251630ACF
:100E8000D8B441EF0DF08251690AD8B4C8EF08F028
:100E900082517A0AD8B4DBEF09F08251490AD8B4FA
:100EA00067EF08F08251500AD8B485EF07F08251FD
:100EB000700AD8B4C8EF07F08251540AD8B4F3EFDF
:100EC00007F08251740AD8B439EF08F08251730ADE
:100ED000D8B4F3EF0AF08251530AD8B458EF0BF0AC
:100EE00076EF0DF0040114EE00F080517F0BE12647
:100EF00082C4E7FF802B12000D0E826F72EC07F0A8
:100F00000A0E826F72EC07F0120083C31EF184C3D5
:100F10001FF185C320F186C321F187C322F188C365
:100F200023F189C324F18AC325F18BC326F18CC335
:100F300027F1010106EC14F07DEC13F0160E0C6E97
:100F400000C10BF0E9EC05F0170E0C6E01C10BF0BF
:100F5000E9EC05F0180E0C6E02C10BF0E9EC05F09F
:100F6000190E0C6E03C10BF0E9EC05F000C15DF148
:100F700001C15EF102C15FF103C160F100C161F125
:100F800001C162F102C163F103C164F167EF08F0CE
:100F900083C31EF184C31FF185C320F186C321F1F1
:100FA00087C322F188C323F189C324F18AC325F1C1
:100FB0008BC326F18CC327F1010106EC14F07DEC04
:100FC00013F000C15DF101C15EF102C15FF103C127
:100FD00060F100C161F101C162F102C163F103C1BD
:100FE00064F167EF08F083C31EF184C31FF185C36A
:100FF00020F186C321F187C322F188C323F189C37D
:1010000024F18AC325F18CC326F18DC327F1010198
:1010100006EC14F07DEC13F00101000E046F000EDD
:10102000056F010E066F000E076FD0EC12F01A0E5E
:101030000C6E00C10BF0E9EC05F01B0E0C6E01C14B
:101040000BF0E9EC05F01C0E0C6E02C10BF0E9ECA4
:1010500005F01D0E0C6E03C10BF0E9EC05F000C1AC
:1010600065F101C166F102C167F103C168F167EF83
:1010700008F083C31EF184C31FF185C320F186C32A
:1010800021F187C322F188C323F189C324F18AC3E4
:1010900025F18CC326F18DC327F1010106EC14F074
:1010A0007DEC13F00101000E046F000E056F010EC0
:1010B000066F000E076FD0EC12F000C165F101C1A0
:1010C00066F102C167F103C168F167EF08F0160E1F
:1010D000FFEC05F0E8CF00F1170EFFEC05F0E8CFCC
:1010E00001F1180EFFEC05F0E8CF02F1190EFFEC4C
:1010F00005F0E8CF03F15BEC13F087EC11F004018D
:10110000730E826F72EC07F004012C0E826F72EC8A
:1011100007F05DC100F15EC101F15FC102F160C184
:1011200003F15BEC13F087EC11F00401730E826F96
:1011300072EC07F004012C0E826F72EC07F01A0EAD
:10114000FFEC05F0E8CF00F11B0EFFEC05F0E8CF57
:1011500001F11C0EFFEC05F0E8CF02F11D0EFFECD3
:1011600005F0E8CF03F191EC0DF004012C0E826F35
:1011700072EC07F065C100F166C101F167C102F1CF
:1011800068C103F191EC0DF07CEC07F076EF0DF007
:101190000401690E826F72EC07F004012C0E826F5D
:1011A00072EC07F00101040E006F000E016F000EDB
:1011B000026F000E036F5BEC13F020C182F4040198
:1011C000300E822772EC07F021C182F40401300E48
:1011D000822772EC07F022C182F40401300E8227CC
:1011E00072EC07F023C182F40401300E822772EC06
:1011F00007F024C182F40401300E822772EC07F05C
:1012000025C182F40401300E822772EC07F026C15A
:1012100082F40401300E822772EC07F027C182F4B9
:101220000401300E822772EC07F004012C0E826F4D
:1012300072EC07F00101030E006F000E016F000E4B
:10124000026F000E036F5BEC13F020C182F4040107
:10125000300E822772EC07F021C182F40401300EB7
:10126000822772EC07F022C182F40401300E82273B
:1012700072EC07F023C182F40401300E822772EC75
:1012800007F024C182F40401300E822772EC07F0CB
:1012900025C182F40401300E822772EC07F026C1CA
:1012A00082F40401300E822772EC07F027C182F429
:1012B0000401300E822772EC07F004012C0E826FBD
:1012C00072EC07F00101130E006F000E016F000EAB
:1012D000026F000E036F5BEC13F020C182F4040177
:1012E000300E822772EC07F021C182F40401300E27
:1012F000822772EC07F022C182F40401300E8227AB
:1013000072EC07F023C182F40401300E822772ECE4
:1013100007F024C182F40401300E822772EC07F03A
:1013200025C182F40401300E822772EC07F026C139
:1013300082F40401300E822772EC07F027C182F498
:101340000401300E822772EC07F004012C0E826F2C
:1013500072EC07F0200EF86EF76AF66A04010900D5
:10136000F5CF82F472EC07F00900F5CF82F472EC4D
:1013700007F00900F5CF82F472EC07F00900F5CF11
:1013800082F472EC07F00900F5CF82F472EC07F0FA
:101390000900F5CF82F472EC07F00900F5CF82F472
:1013A00072EC07F00900F5CF82F472EC07F07CECE8
:1013B00007F076EF0DF08351630AD8A476EF0DF0B5
:1013C0008451610AD8A476EF0DF085516C0AD8A437
:1013D00076EF0DF08651410A42E08651440A1BE047
:1013E0008651420AD8B442EF0AF08651350AD8B481
:1013F00000EF0FF08651360AD8B455EF0FF0865142
:10140000370AD8B4BEEF0FF08651380AD8B41CEFB3
:1014100010F076EF0DF00798079A04017A0E826FAC
:1014200072EC07F00401780E826F72EC07F0040191
:10143000640E826F72EC07F081A826EF0AF00401B7
:10144000550E826F72EC07F02BEF0AF004014C0E80
:10145000826F72EC07F07CEC07F076EF0DF00788F6
:10146000079A04017A0E826F72EC07F00401410EB4
:10147000826F72EC07F00401610E826F72EC07F06C
:101480001CEF0AF00798078A04017A0E826F72EC4B
:1014900007F00401420E826F72EC07F00401610E46
:1014A000826F72EC07F01CEF0AF00101620E046F0C
:1014B000010E056F000E066F000E076F59C100F197
:1014C0005AC101F15BC102F15CC103F1C1EC12F040
:1014D00003BFB2EF0AF00E0EFFEC05F0E8CF0CF1FF
:1014E0000F0EFFEC05F0E8CF0DF1100EFFEC05F04C
:1014F000E8CF0EF1110EFFEC05F0E8CF0FF10AEC8A
:1015000012F059C104F15AC105F15BC106F15CC189
:1015100007F1C1EC12F00782CEEC11F00AEC12F0E8
:101520000792CEEC11F059C100F15AC101F15BC133
:1015300002F15CC103F10792CEEC11F0CC0E046F06
:10154000E00E056F870E066F050E076FC1EC12F0F7
:1015500000C10CF101C10DF102C10EF103C10FF187
:10156000EAEF0AF00101800E006F1A0E016F060EFD
:10157000026F000E036F42C104F143C105F144C183
:1015800006F145C107F1C1EC12F003AFCBEF0AF051
:10159000B8EC13F012000E0EFFEC05F0E8CF0CF1E2
:1015A0000F0EFFEC05F0E8CF0DF1100EFFEC05F08B
:1015B000E8CF0EF1110EFFEC05F0E8CF0FF142C1BC
:1015C00000F143C101F144C102F145C103F10782B9
:1015D000CEEC11F00CC100F10DC101F10EC102F110
:1015E0000FC103F112000401730E826F72EC07F059
:1015F00004012C0E826F72EC07F0078455C159F17B
:1016000056C15AF157C15BF158C15CF13EC142F17C
:101610003FC143F140C144F141C145F14AC14CF1E0
:101620004BC14DF1079419EC0BF07CEC07F076EF11
:101630000DF059C100F15AC101F15BC102F15CC169
:1016400003F101015BEC13F087EC11F00401630E70
:10165000826F72EC07F004012C0E826F72EC07F0BF
:1016600042C100F143C101F144C102F145C103F19E
:1016700001015BEC13F087EC11F00401660E826F40
:1016800072EC07F004012C0E826F72EC07F0B8ECDC
:1016900013F04CC100F14DC101F101015BEC13F0FD
:1016A00087EC11F00401740E826F72EC07F01200E7
:1016B0000F820401530E826F72EC07F004012C0EAE
:1016C000826F72EC07F083C31EF184C31FF185C3E0
:1016D00020F186C321F187C322F188C323F189C396
:1016E00024F18AC325F18BC326F18CC327F10101B4
:1016F00006EC14F07DEC13F000C159F101C15AF170
:1017000002C15BF103C15CF18EC31EF18FC31FF1F7
:1017100090C320F191C321F192C322F193C323F12D
:1017200094C324F195C325F196C326F197C327F1FD
:10173000010106EC14F07DEC13F000C142F101C18F
:1017400043F102C144F103C145F1F9EC13F099C32F
:1017500023F19AC324F19BC325F19CC326F19DC3B9
:1017600027F1010106EC14F07DEC13F000C14CF1FF
:1017700001C14DF119EC0BF004012C0E826F72ECDB
:1017800007F0CAEF0BF08251520A03E10E82CAEF52
:101790000BF00E9207840FB2E2EF0BF055C159F136
:1017A00056C15AF157C15BF158C15CF13EC142F1DB
:1017B0003FC143F140C144F141C145F14AC14CF13F
:1017C0004BC14DF107940EA004EF0CF001016567C9
:1017D000F1EF0BF06667F1EF0BF06767F1EF0BF0DD
:1017E0006867F5EF0BF004EF0CF055EC0AF065C1FB
:1017F00004F166C105F167C106F168C107F1C1ECEA
:1018000012F003BF3EEF0DF055EC0AF00101000E9F
:10181000046F000E056F010E066F000E076FEFECF0
:1018200012F00401720E826F72EC07F004012C0EAC
:10183000826F72EC07F05BEC13F01D6725EF0CF084
:101840000401200E826F28EF0CF004012D0E826F30
:1018500072EC07F024C182F40401300E822772EC8E
:1018600007F025C182F40401300E822772EC07F0E4
:1018700004012E0E826F72EC07F026C182F404017F
:10188000300E822772EC07F027C182F40401300E7B
:10189000822772EC07F004016D0E826F72EC07F084
:1018A00004012C0E826F72EC07F042C100F143C1BB
:1018B00001F144C102F145C103F101015BEC13F0F8
:1018C00087EC11F00401480E826F72EC07F00401FE
:1018D0007A0E826F72EC07F004012C0E826F72ECAC
:1018E00007F059C100F15AC101F15BC102F15CC1BD
:1018F00003F101015BEC13F087EC11F00401630EBE
:10190000826F72EC07F004012C0E826F72EC07F00C
:1019100059C100F15AC101F15BC102F15CC103F18F
:1019200001010A0E046F000E056F000E066F000E17
:10193000076FD0EC12F0000E046F120E056F000E50
:10194000066F000E076FEFEC12F05BEC13F01EC198
:1019500082F40401300E822772EC07F01FC182F47A
:101960000401300E822772EC07F020C182F40401DA
:10197000300E822772EC07F021C182F40401300E90
:10198000822772EC07F022C182F40401300E822714
:1019900072EC07F023C182F40401300E822772EC4E
:1019A00007F024C182F40401300E822772EC07F0A4
:1019B00004012E0E826F72EC07F025C182F404013F
:1019C000300E822772EC07F026C182F40401300E3B
:1019D000822772EC07F027C182F40401300E8227BF
:1019E00072EC07F00401730E826F72EC07F00401D1
:1019F0002C0E826F72EC07F0B8EC13F04CC100F1C2
:101A00004DC101F1A0EC0EF00EB20AEF0DF00EA0E8
:101A10003CEF0DF004012C0E826F72EC07F0200EEB
:101A2000F86EF76AF66A04010900F5CF82F472ECE9
:101A300007F00900F5CF82F472EC07F00900F5CF4A
:101A400082F472EC07F00900F5CF82F472EC07F033
:101A50000900F5CF82F472EC07F00900F5CF82F4AB
:101A600072EC07F00900F5CF82F472EC07F0090080
:101A7000F5CF82F472EC07F07CEC07F00E9076EF75
:101A80000DF00401630E826F72EC07F004012C0E5E
:101A9000826F72EC07F07CEC0DF004012C0E826F6B
:101AA00072EC07F0EFEC0DF004012C0E826F72EC7B
:101AB00007F06BEC0EF004012C0E826F72EC07F055
:101AC0000101F80E006FCD0E016F660E026F030E5E
:101AD000036F91EC0DF004012C0E826F72EC07F095
:101AE00081EC0EF07CEC07F076EF0DF00301A26BB9
:101AF00007900F9285EF10F0D8900E0EFFEC05F0D6
:101B0000E8CF00F10F0EFFEC05F0E8CF01F1100E69
:101B1000FFEC05F0E8CF02F1110EFFEC05F0E8CF85
:101B200003F10101000E046F000E056F010E066F38
:101B3000000E076FEFEC12F05BEC13F01EC182F4A5
:101B40000401300E822772EC07F01FC182F40401F9
:101B5000300E822772EC07F020C182F40401300EAF
:101B6000822772EC07F021C182F40401300E822733
:101B700072EC07F022C182F40401300E822772EC6D
:101B800007F023C182F40401300E822772EC07F0C3
:101B900024C182F40401300E822772EC07F025C1C3
:101BA00082F40401300E822772EC07F004012E0E3D
:101BB000826F72EC07F026C182F40401300E822796
:101BC00072EC07F027C182F40401300E822772EC18
:101BD00007F004016D0E826F72EC07F01200120E16
:101BE000FFEC05F0E8CF00F1130EFFEC05F0E8CFB5
:101BF00001F1140EFFEC05F0E8CF02F1150EFFEC39
:101C000005F0E8CF03F101010A0E046F000E056F25
:101C1000000E066F000E076FD0EC12F0000E046F7E
:101C2000120E056F000E066F000E076FEFEC12F03C
:101C30005BEC13F01EC182F40401300E822772ECBB
:101C400007F01FC182F40401300E822772EC07F006
:101C500020C182F40401300E822772EC07F021C10A
:101C600082F40401300E822772EC07F022C182F464
:101C70000401300E822772EC07F023C182F40401C4
:101C8000300E822772EC07F024C182F40401300E7A
:101C9000822772EC07F004012E0E826F72EC07F0BF
:101CA00025C182F40401300E822772EC07F026C1B0
:101CB00082F40401300E822772EC07F027C182F40F
:101CC0000401300E822772EC07F00401730E826F5C
:101CD00072EC07F012000A0EFFEC05F0E8CF00F1FD
:101CE0000B0EFFEC05F0E8CF01F10C0EFFEC05F058
:101CF000E8CF02F10D0EFFEC05F0E8CF03F1A0EF05
:101D00000EF0060EFFEC05F0E8CF00F1070EFFEC39
:101D100005F0E8CF01F1080EFFEC05F0E8CF02F185
:101D2000090EFFEC05F0E8CF03F1A0EF0EF0010182
:101D3000B8EC13F007844AC100F14BC101F10794DC
:101D40000101E80E046F800E056F000E066F000E95
:101D5000076FD0EC12F0000E046F040E056F000E3A
:101D6000066F000E076FEFEC12F0880E046F130E73
:101D7000056F000E066F000E076FC1EC12F00A0E21
:101D8000046F000E056F000E066F000E076FEFEC7C
:101D900012F05BEC13F001011D67D4EF0EF00401AB
:101DA000200E826FD7EF0EF004012D0E826F72ECC1
:101DB00007F024C182F40401300E822772EC07F090
:101DC00025C182F40401300E822772EC07F026C18F
:101DD00082F40401300E822772EC07F004012E0E0B
:101DE000826F72EC07F027C182F40401300E822763
:101DF00072EC07F00401430E826F72EC07F01200E0
:101E000087C31EF188C31FF189C320F18AC321F162
:101E10008BC322F18CC323F18DC324F18EC325F132
:101E200090C326F191C327F101011D6B06EC14F05C
:101E30007DEC13F00101000E046F000E056F010E22
:101E4000066F000E076FD0EC12F00E0E0C6E00C184
:101E50000BF0E9EC05F00F0E0C6E01C10BF0E9EC94
:101E600005F0100E0C6E02C10BF0E9EC05F0110E3E
:101E70000C6E03C10BF0E9EC05F004017A0E826FE1
:101E800072EC07F004012C0E826F72EC07F0040173
:101E9000350E826F72EC07F004012C0E826F72EC2B
:101EA00007F07CEC0DF02BEF0AF087C31EF188C31E
:101EB0001FF189C320F18AC321F18BC322F18CC3A6
:101EC00023F18DC324F18EC325F190C326F191C374
:101ED00027F101011D6B06EC14F07DEC13F0880E68
:101EE000046F130E056F000E066F000E076FC5EC32
:101EF00012F0000E046F040E056F000E066F000E48
:101F0000076FD0EC12F00101E80E046F800E056F30
:101F1000000E066F000E076FEFEC12F00A0E0C6E4B
:101F200000C10BF0E9EC05F00B0E0C6E01C10BF0DB
:101F3000E9EC05F00C0E0C6E02C10BF0E9EC05F0BB
:101F40000D0E0C6E03C10BF0E9EC05F004017A0EE6
:101F5000826F72EC07F004012C0E826F72EC07F0B6
:101F60000401360E826F72EC07F004012C0E826FB2
:101F700072EC07F06BEC0EF02BEF0AF087C31EF14A
:101F800088C31FF189C320F18AC321F18BC322F1D9
:101F90008CC323F18DC324F18FC325F190C326F1A7
:101FA00091C327F1010106EC14F07DEC13F0000E53
:101FB000046F120E056F000E066F000E076FD0EC57
:101FC00012F001010A0E046F000E056F000E066F7D
:101FD000000E076FEFEC12F0120E0C6E00C10BF04A
:101FE000E9EC05F0130E0C6E01C10BF0E9EC05F005
:101FF000140E0C6E02C10BF0E9EC05F0150E0C6E20
:1020000003C10BF0E9EC05F004017A0E826F72EC6B
:1020100007F004012C0E826F72EC07F00401370EFA
:10202000826F72EC07F004012C0E826F72EC07F0E5
:10203000EFEC0DF02BEF0AF087C31EF188C31FF100
:1020400089C320F18AC321F18BC322F18CC323F110
:102050008DC324F18EC325F190C326F191C327F1DE
:1020600001011D6B06EC14F07DEC13F0880E046F7B
:10207000130E056F000E066F000E076FC5EC12F011
:10208000000E046F040E056F000E066F000E076F42
:10209000D0EC12F00101E80E046F800E056F000E07
:1020A000066F000E076FEFEC12F0060E0C6E00C10B
:1020B0000BF0E9EC05F0070E0C6E01C10BF0E9EC3A
:1020C00005F0080E0C6E02C10BF0E9EC05F0090EEC
:1020D0000C6E03C10BF0E9EC05F004017A0E826F7F
:1020E00072EC07F004012C0E826F72EC07F0040111
:1020F000380E826F72EC07F004012C0E826F72ECC6
:1021000007F081EC0EF02BEF0AF081A843EF11F0FD
:1021100007A8FCEF10F00101800E006F1A0E016F8E
:10212000060E026F000E036F3EC104F13FC105F1C0
:1021300040C106F141C107F1C1EC12F003BF43EF0A
:1021400011F081EC11F03EC100F13FC101F140C13D
:1021500002F141C103F10782CEEC11F00CC104F190
:102160000DC105F10EC106F10FC107F1F80E006FA8
:10217000CD0E016F660E026F030E036FC1EC12F0FD
:102180000E0E0C6E00C10BF0E9EC05F00F0E0C6E9C
:1021900001C10BF0E9EC05F0100E0C6E02C10BF062
:1021A000E9EC05F0110E0C6E03C10BF0E9EC05F043
:1021B00007840101B8EC13F04AC100F14BC101F1F1
:1021C00007940A0E0C6E00C10BF0E9EC05F00B0E43
:1021D0000C6E01C10BF0E9EC05F00C0E0C6E02C1A7
:1021E0000BF0E9EC05F00D0E0C6E03C10BF0E9EC01
:1021F00005F0079843EF11F007AA43EF11F00784A9
:102200000101B8EC13F04AC100F14BC101F1079490
:10221000060E0C6E00C10BF0E9EC05F0070E0C6E1B
:1022200001C10BF0E9EC05F0080E0C6E02C10BF0D9
:10223000E9EC05F0090E0C6E03C10BF0E9EC05F0BA
:10224000078455C100F156C101F157C102F158C1CF
:1022500003F10794120E0C6E00C10BF0E9EC05F0CF
:10226000130E0C6E01C10BF0E9EC05F0140E0C6EB0
:1022700002C10BF0E9EC05F0150E0C6E03C10BF07A
:10228000E9EC05F0079A0401805181197F0B0BE0FE
:102290009EA809D014EE00F081517F0BE126E75093
:1022A000812B0F01AD6EEDEF06F00CC100F10DC1F9
:1022B00001F10EC102F10FC103F1000E046F000E17
:1022C000056F010E066F000E076FEFEC12F01DA1F7
:1022D00080EF11F01451D8B480EF11F00CC100F16F
:1022E0000DC101F10EC102F10FC103F1000E046F27
:1022F000000E056F0A0E066F000E076FEFEC12F06E
:10230000120001010C6B0D6B0E6B0F6B12001EC1E6
:1023100082F40401300E822772EC07F01FC182F4B0
:102320000401300E822772EC07F020C182F4040110
:10233000300E822772EC07F021C182F40401300EC6
:10234000822772EC07F022C182F40401300E82274A
:1023500072EC07F023C182F40401300E822772EC84
:1023600007F024C182F40401300E822772EC07F0DA
:1023700025C182F40401300E822772EC07F026C1D9
:1023800082F40401300E822772EC07F027C182F438
:102390000401300E822772EC07F012000101005395
:1023A00005E1015303E1025301E1002B91EC12F02E
:1023B000B8EC13F02C51006F2D51016F420E046FD9
:1023C0004B0E056F000E066F000E076FD0EC12F07B
:1023D00000C104F101C105F102C106F103C107F119
:1023E0000CC100F10DC101F10EC102F10FC103F1E9
:1023F00007B2FFEF11F0C5EC12F001EF12F0C1ECE3
:1024000012F000C10CF101C10DF102C10EF103C1C6
:102410000FF11200B8EC13F04CC100F14DC101F105
:10242000060EFFEC05F0E8CF04F1070EFFEC05F017
:10243000E8CF05F1080EFFEC05F0E8CF06F1090E34
:10244000FFEC05F0E8CF07F1C1EC12F000C118F184
:1024500001C119F102C11AF103C11BF1290E046F68
:10246000000E056F000E066F000E076FD0EC12F025
:10247000EE0E046F430E056F000E066F000E076F21
:10248000C5EC12F018C104F119C105F11AC106F129
:102490001BC107F1D0EC12F000C110F101C111F124
:1024A00002C112F103C113F1120EFFEC05F0E8CFE7
:1024B00004F1130EFFEC05F0E8CF05F1140EFFEC6C
:1024C00005F0E8CF06F1150EFFEC05F0E8CF07F1B7
:1024D0000D0E006F000E016F000E026F000E036FF5
:1024E000D0EC12F0180E046F000E056F000E066F90
:1024F000000E076FEFEC12F010C104F111C105F1ED
:1025000012C106F113C107F1C5EC12F06A0E046F97
:102510002A0E056F000E066F000E076FC1EC12F059
:102520001200BF0EFA6E200E2D6F2C6BD890003764
:10253000013702370337D8B0A2EF12F02D2F97EFF3
:1025400012F02C072D070353D8B412000331070BE8
:102550008009326F03390F0B010F2C6F80EC5FF095
:10256000336F2C0580EC5FF0335D335F2C6B3233BF
:10257000D8B02C272C3332A9B7EF12F033512C27C7
:102580001200DDEC13F0D8B0120003510719286FC8
:10259000A0EC13F0D8900751031928AF800F120058
:1025A000286BC4EC13F0D8A0DAEC13F0D8B012000A
:1025B000AFEC13F0B8EC13F01F0E296FF0EC13F032
:1025C0000B35D8B0A0EC13F0D8A00335D8B012006A
:1025D000292FDEEF12F028B1C7EC13F01200286BA0
:1025E00004510511061107110008D8A0C4EC13F01E
:1025F000D8A0DAEC13F0D8B01200086B096B0A6BA4
:102600000B6BF0EC13F01F0E296FF0EC13F0075179
:102610000B5DD8A418EF13F006510A5DD8A418EF8B
:1026200013F00551095DD8A418EF13F00451085DAB
:10263000D8A02BEF13F00451085F0551D8A0053D39
:10264000095F0651D8A0063D0A5F0751D8A0073D93
:102650000B5FD8900081292F05EF13F028B1C7EC4C
:1026600013F0286BC4EC13F0D890F4EC13F007517E
:102670000B5DD8A448EF13F006510A5DD8A448EFCB
:1026800013F00551095DD8A448EF13F00451085D1B
:10269000D8A057EF13F0003F57EF13F0013F57EF6B
:1026A00013F0023F57EF13F0032BD8B4120028B1F8
:1026B000C7EC13F012000101286BC4EC13F0D8B082
:1026C0001200F9EC13F0200E296F003701370237A2
:1026D000033711EE27F00A0E2A6FE7360A0EE75C81
:1026E000D8B0E76EE5522A2F6DEF13F0292F65EF72
:1026F00013F028B11D81D890120001010A0E286F35
:10270000200E296F11EE1DF028512A6F0A0ED89065
:10271000E652D8B0E726E7322A2F88EF13F00333CA
:10272000023301330033292F82EF13F0E750FF0FFC
:10273000D8A00335D8B012001DB1C7EC13F01200B9
:10274000045100270551D8B0053D01270651D8B0E6
:10275000063D02270751D8B0073D0327120000515C
:10276000086F0151096F02510A6F03510B6F12007C
:102770000101006B016B026B036B12000101046B22
:10278000056B066B076B12000335D8A012000351CE
:10279000800B001F011F021F031F003FD7EF13F024
:1027A000013FD7EF13F0023FD7EF13F0032B282B95
:1027B000032512000735D8A012000751800B041F13
:1027C000051F061F071F043FEDEF13F0053FEDEF58
:1027D00013F0063FEDEF13F0072B282B072512000F
:1027E0000037013702370337083709370A370B3705
:1027F000120001011D6B1E6B1F6B206B216B226B86
:10280000236B246B256B266B276B12001E510F0B5D
:102810001E6F1F510F0B1F6F20510F0B206F215187
:102820000F0B216F22510F0B226F23510F0B236FC0
:1028300024510F0B246F25510F0B256F26510F0BC1
:0A284000266F27510F0B276F1200BF
:10BF0000E844F926000C160C2B0C3F0C520C640C68
:10BF1000760C860C960CA50CB30CC10CCF0CDC0C6B
:06BF2000E80CF40C000C1B
:00000001FF
